:100000000EC015C014C013C012C011C010C00FC064
:100010000EC00DC00CC00BC00AC009C008C011241E
:100020001FBECFE5D2E0DEBFCDBF1AD037C0E8CFCC
:100030000F931F9300E010E0980106171707280799
:10004000390759F0EFECF7E03197F1F700C0000005
:100050000F5F1F4F2F4F3F4FF0CF1F910F9108950C
:10006000F89480E886BD16BC80E681BF80E187BB3E
:1000700090E18AE098BB18BA8150E1F785ED8A9546
:10008000F1F700008AE098BB18BA8150E1F7EFE180
:10009000FEE43197F1F700C00000EBCFF894FFCFFA
:00000001FF
